:020000040800F2
:1000000000070020F5040008F1260008A9260008D2
:10001000D1260008A9260008C9260008F704000810
:10002000F7040008F7040008F7040008E5360008A4
:10003000F7040008F7040008F7040008F7040008B4
:10004000F7040008F7040008F7040008F7040008A4
:10005000F7040008F7040008F144000819450008F7
:10006000414500086945000891450008F70400086B
:10007000F7040008F7040008F7040008F704000874
:10008000F7040008F7040008F70400085D260008DC
:100090008926000899260008F7040008B9450008D9
:1000A000F7040008F7040008F7040008F704000844
:1000B000B5460008F7040008F7040008F704000834
:1000C000F7040008F7040008F7040008F704000824
:1000D000F70400088D460008A1460008F704000850
:1000E0001D460008F7040008F7040008F70400089C
:1000F000F7040008F7040008F7040008F7040008F4
:10010000F7040008F7040008F7040008F7040008E3
:10011000F7040008F7040008F7040008F7040008D3
:10012000F7040008F7040008F7040008F7040008C3
:10013000F7040008F7040008F7040008F7040008B3
:10014000F7040008F7040008F7040008F7040008A3
:10015000F7040008F7040008F7040008F704000893
:10016000F7040008F7040008F7040008F704000883
:10017000F7040008F7040008F7040008F704000873
:10018000F7040008F7040008F7040008F704000863
:10019000F7040008F7040008F7040008F704000853
:1001A000F7040008F7040008F7040008F704000843
:1001B000F7040008F7040008F7040008F704000833
:1001C000F7040008F7040008F7040008F704000823
:1001D000F7040008F7040008F7040008F704000813
:1001E000CD12000800000000000000000000000028
:1001F00053B94AB9002908BF00281CBF4FF0FF318E
:100200004FF0FF3000F074B9ADF1080C6DE904CE89
:1002100000F006F8DDF804E0DDE9022304B07047E1
:100220002DE9F047089D04468E46002B4DD18A42A9
:10023000944669D9B2FA82F252B101FA02F3C2F1DC
:10024000200120FA01F10CFA02FC41EA030E94406D
:100250004FEA1C48210CBEFBF8F61FFA8CF708FB8E
:1002600016E341EA034306FB07F199420AD91CEB66
:10027000030306F1FF3080F01F81994240F21C8198
:10028000023E63445B1AA4B2B3FBF8F008FB1033E0
:1002900044EA034400FB07F7A7420AD91CEB040415
:1002A00000F1FF3380F00A81A74240F207816444E5
:1002B000023840EA0640E41B00261DB1D44000236A
:1002C000C5E900433146BDE8F0878B4209D9002DCE
:1002D00000F0EF800026C5E9000130463146BDE858
:1002E000F087B3FA83F6002E4AD18B4202D38242C2
:1002F00000F2F980841A61EB030301209E46002D71
:10030000E0D0C5E9004EDDE702B9FFDEB2FA82F2C5
:10031000002A40F09280A1EB0C014FEA1C471FFA23
:100320008CFE0126200CB1FBF7F307FB131140EA0A
:1003300001410EFB03F0884208D91CEB010103F1D7
:10034000FF3802D2884200F2CB804346091AA4B299
:10035000B1FBF7F007FB101144EA01440EFB00FE6D
:10036000A64508D91CEB040400F1FF3102D2A645D2
:1003700000F2BB800846A4EB0E0440EA03409CE771
:10038000C6F12007B34022FA07FC4CEA030C20FA1E
:1003900007F401FA06F31C43F9404FEA1C4900FA3E
:1003A00006F3B1FBF9F8200C1FFA8CFE09FB1811BB
:1003B00040EA014108FB0EF0884202FA06F20BD92E
:1003C0001CEB010108F1FF3A80F08880884240F27E
:1003D0008580A8F102086144091AA4B2B1FBF9F0C2
:1003E00009FB101144EA014100FB0EFE8E4508D9BD
:1003F0001CEB010100F1FF346CD28E456AD9023842
:10040000614440EA0840A0FB0294A1EB0E01A14226
:10041000C846A64656D353D05DB1B3EB080261EB94
:100420000E0101FA07F722FA06F3F1401F43C5E96E
:10043000007100263146BDE8F087C2F12003D840A4
:100440000CFA02FC21FA03F3914001434FEA1C47E6
:100450001FFA8CFEB3FBF7F007FB10360B0C43EAD8
:10046000064300FB0EF69E4204FA02F408D91CEB88
:10047000030300F1FF382FD29E422DD90238634486
:100480009B1B89B2B3FBF7F607FB163341EA034126
:1004900006FB0EF38B4208D91CEB010106F1FF3875
:1004A00016D28B4214D9023E6144C91A46EA00466C
:1004B00038E72E46284605E70646E3E61846F8E6FE
:1004C0004B45A9D2B9EB020864EB0C0E0138A3E747
:1004D0004646EAE7204694E74046D1E7D0467BE728
:1004E000023B614432E7304609E76444023842E7A0
:1004F000704700BF02E000F000F8FEE772B6374830
:1005000080F30888364880F3098836483649086001
:1005100040F20000CCF200004EF63471CEF2000141
:100520000860BFF34F8FBFF36F8F40F20000C0F23F
:10053000F0004EF68851CEF200010860BFF34F8FF5
:10054000BFF36F8F4FF00000E1EE100A4EF63C71E2
:10055000CEF200010860062080F31488BFF36F8F8D
:1005600003F0D0FD03F062FE4FF055301F491B4AE7
:1005700091423CBF41F8040BFAE71D49184A9142E9
:100580003CBF41F8040BFAE71A491B4A1B4B9A423D
:100590003EBF51F8040B42F8040BF8E7002018495D
:1005A000184A91423CBF41F8040BFAE703F0AEFD54
:1005B00003F08AFE144C154DAC4203DA54F8041BC8
:1005C0008847F9E700F042F8114C124DAC4203DACB
:1005D00054F8041B8847F9E703F096BD0007002094
:1005E000002300200000000808ED00E000010020CA
:1005F00000070020F04F0008002300208023002087
:100600008023002030520020E0010008E4010008AF
:10061000E4010008E40100082DE9F04F2DED108AF7
:10062000C1F80CD0C3689D46BDEC108ABDE8F08FC0
:10063000002383F311882846A047002003F0D4F953
:10064000FEE703F037F900DFFEE70000F8B500F041
:100650004FFE03F0F1FC074603F040FD054600287D
:100660003FD12C4B9F423CD001339F423CD02A4B80
:1006700027F0FF029A423AD1F8B200F045FC2E462C
:1006800042F2107400F046FC08B10024264601F046
:100690001DF980B3032000F045F80024264635B14B
:1006A0001E4B9F4203D003F011FD0024264600207C
:1006B00003F0CCFC1A4B1B691B0722D40EB100F0CF
:1006C00047F800F093FC00F015FE02F019F805461B
:1006D000CCB102F015F8401BA04214D900F038F854
:1006E000F3E72E460024CDE704460126CAE7064676
:1006F0004FF47A74C6E7002CD1D04FF47A740126F7
:10070000CDE70024DDE700F0B9FC4FF47A7003F088
:1007100071F9DDE7010007B0000008B0263A09B022
:1007200000040240084B187003280CD8DFE800F0E2
:1007300008050208022000F03BBE022000F02EBE99
:10074000024B00225A60704780230020842300203F
:1007500010B501F0BBF830B1204B03221A70204BCA
:1007600000225A6010BD1F4B1F4A1C4619680131F8
:10077000F8D004339342F9D162681C4B9A42F1D904
:100780001B4B9B6803F1006303F580339A42E9D267
:1007900003F070FC03F082FC002000F0C5FD022095
:1007A000FFF7C0FF134B1A6C00221A64196E1A6609
:1007B000196E596C5A64596E5A665B6E72B64FF078
:1007C000E0233021C3F8084DD4E9003281F31188C9
:1007D0009D4683F308881047C4E700BF80230020AC
:1007E000842300200000010820000108FFFF00080A
:1007F0000023002000380240094A136849F26900CA
:1008000099B21B0C00FB01331360064B186844F2CD
:10081000506182B2000C01FB0200186080B2704788
:10082000182300201423002010B5002110220446B4
:1008300000F0DAFD034B03CB206061601868A06014
:1008400010BD00BF107AFF1F2DE9F041ADF54E7DC0
:100850000DF134086CAC40F2751207460D460EA837
:100860000021C8F8001000F0BFFD4FF4C472002151
:10087000204600F0B9FD01F043FF274B4FF47A7298
:10088000B0FBF2F0186093E80700022384E8070049
:100890000DF5E9702382FFF7C7FF4EF603131F49DA
:1008A000238407A804F0AAFA162384F832310DF243
:1008B000E32207AB0DF12C0C1E4603CE66451060FB
:1008C0005160334602F10802F6D130681060B388F7
:1008D000938041460122204600F0D2FD002303937D
:1008E000AB7E029305F11903019380B20123CDE998
:1008F00004800093E97E06A3D3E90023384602F082
:10090000C7FA0DF54E7DBDE8F08100BFAFF3008062
:100910009E6AC421818A46EE8C2300200C4E00087A
:100920002DE9F0412C4C237ADAB080460D465BBBB2
:1009300027A9284600F0B4FE0746002842D19DF8BA
:100940009D60C82E3ED801464FF4A662204600F0B6
:100950004BFD4FF48073C4F8F8314FF40073C4F8C2
:100960000C334FF44073C4F8203432460DF19E012D
:1009700004F1090000F026FD26449DF89C307772B2
:1009800023720BB9EB7E23728122002106AC27A8CB
:1009900000F02AFD0122214627A800F0BDFE002319
:1009A0000393AB7E029305F1190380B201932823D0
:1009B000CDE904400093E97E05A3D3E90023404636
:1009C00002F066FA5AB0BDE8F08100BFAFF30080D4
:1009D00026417272DF25D7B7A8440020F0B5254E16
:1009E0004FF48A7505FB0065F1B096F8D83085F8AC
:1009F000DC300024D822214685F8E8403AA800F0EF
:100A0000F3FC06F1090000F0E7FCD5F8E4308DF8BE
:100A1000F000C2B206AF06F109010DF1F100CDE917
:100A20003A3400F0CFFC394601223AA800F0A0FE8B
:100A300080B2CDE9047008230127CDE9023706F121
:100A4000D803019330230093317A0B4807A3D3E9ED
:100A5000002302F01DFAA04206DD01F051FEC5F8A8
:100A6000E000384671B0F0BD2046FBE778F6339FD2
:100A700093CACD8DA8440020A43300202DE9F04175
:100A80001D4D1E4E1E4F86B0284602F02DFA03461D
:100A900058B30024CDE90344ADF81440027B8DF82F
:100AA000142099684068029403AA03C21B68DFF807
:100AB000548043F00043029301F024FE821941F177
:100AC0000003009402A9384601F0E6F8A04205DDD3
:100AD000284602F00DFA88F80040D5E798F8003073
:100AE000072B05D8013388F8003006B0BDE8F08147
:100AF000014802F0FDF9F8E7A433002040420F005E
:100B0000D8330020DD49002070B50D4614461E463E
:100B100002F01AF950B9022E10D1012C0ED112A3F5
:100B2000D3E90023C5E90023012007E0282C10D0D9
:100B300005D8012C09D0052C0FD0002070BD302C19
:100B4000FBD10BA3D3E90023ECE70BA3D3E90023EC
:100B5000E8E70BA3D3E90023E4E70BA3D3E90023E1
:100B6000E0E700BFAFF30080401DA12026812A0BE3
:100B700078F6339F93CACD8D9E6AC421818A46EE52
:100B800026417272DF25D7B7F017304A39059E56D5
:100B900038B505460E4C0021013500F0E7FBA4F8FE
:100BA0002C55B4F82C0500F0C9FB78B1B4F82C052D
:100BB00000F0D4FB014648B9B4F82C0500F0D6FB90
:100BC000B4F82C350133A4F82C35EAE738BD00BF62
:100BD000A844002010B50A4B0A4A1A6003F5805356
:100BE00093F860203AB9DC6D2CB1204600F0ECFEA1
:100BF000204604F043F8BDE81040034800F0E4BE8E
:100C0000D8330020604E0008204400202DE9F04F2A
:100C10008FB000AF05460C4602F096F8002849D187
:100C2000237E022B1BD1E38A012B18D101F068FD32
:100C30000646FFF7E1FD03464FF4C870DFF8C482B3
:100C4000B3FBF0F206F5167602FB103316FA83F3C7
:100C5000C8F80030E37E33B9A34B00221A703C374A
:100C6000BD46BDE8F08F07F12401204600F0D6FC18
:100C70000028F4D107F11400FFF7D6FD97F82640BD
:100C800007F11401224607F1270004F041F800287B
:100C9000E2D10F2C08D8944B1C70D8F80030A3F583
:100CA0001673C8F80030DAE797F82410284602F0E7
:100CB00043F8D4E7E38A282B2BD010D8012B23D07C
:100CC000052BCCD1BFF34F8F8849894BCA6802F4FA
:100CD000E0621343CB60BFF34F8F00BFFDE7302BC3
:100CE000BDD1844EE17E327A9142B8D1607E3146E8
:100CF000002291F8DC50854200F0A5800132042AE0
:100D000001F58A71F5D1AAE721462846FFF79CFD37
:100D1000A5E721462846FFF703FEA0E7B2F8EC500E
:100D20007B6005F103094FEA99094FEA8902D11D59
:100D3000C908A8EBC1039D46EB460021584600F0C8
:100D400053FB04F1EE012A463144584600F03AFBC9
:100D50007B6813B9012000F0E7FA96F8D20000F0A2
:100D6000EDFA044630B9307200F008FB204600F07E
:100D7000DBFAB1E0D6F8D4203AB996F8D200B6F84A
:100D80002C25824201D8FFF703FFD6F8D4202A444D
:100D9000944208D296F8D200B6F82C25013082424F
:100DA00001D8FFF7F5FE70685FFA89F2594600F046
:100DB00023FB08B9C54679E0726896F8D2002A4448
:100DC0007260D6F8D42005EB0209C6F8D49000F082
:100DD000B5FA814509D396F8D220D6F8D40001326D
:100DE000001B86F8D220C6F8D400FF2D0FD80024AF
:100DF000347200F0C3FA204600F096FA00F066FD67
:100E00003D4B188108B9FFF7A3FCC54627E7BB682F
:100E100096F8D9000AFB0362FB68D2F8E41082F866
:100E2000E83001F58061C2F8E030C2F8E410FFF765
:100E3000D5FDFFF723FE96F8D920013202F0030218
:100E400086F8D920B6E74FF48A7A0AFB02F505F155
:100E5000EA013144204600F0B7FCF86000287FF436
:100E6000FEAE3544012285F8E82001F049FCD5F8B2
:100E7000E020D6ED007ADFED216A801A192838BF0C
:100E8000192040F6B832904228BF1046B8EE677A73
:100E900007EE900AF8EEE77A67EEA67ADFED186AB9
:100EA000E7EE267AFCEEE77AC6ED007A96F8D930BE
:100EB000BB60BA6873680AFB02F4321992F8E81052
:100EC00059B1D2F8E4108B42E8463FF427AF002135
:100ED00082F8E810C2F8E010C5467368064A9B0A1B
:100EE00001331381BBE600BF9D33002000ED00E01D
:100EF0000400FA05A84400208C230020CDCCCC3D72
:100F00006666663FA0330020014B1870704700BF33
:100F10009823002030B54FF000542B4B22689A42A2
:100F200085B007D003F0E4F8044620BB0024204637
:100F300005B030BD254B627D25481A70237D0372B4
:100F40004FF48073C0F8F8314FF40073C0F80C33DD
:100F500000254FF44073C0F820341E49C0F8E45017
:100F6000C922093000F02EFA2046E022294600F07E
:100F70003BFA0124DBE7184A184D136C43F0007369
:100F80001364AA6D164B9A42D0D12B6E013B7E2B77
:100F9000CCD8144A07CA01AB83E8070018460321DE
:100FA00000F062FC6B6D83424FF00003BED12A6DEE
:100FB0008A4201BFAB65054B2A6E1A7003BF0A4B0C
:100FC000EA6D1A601C46B2E79AAD44C5982300202A
:100FD000A8440020160000200038024000660040AF
:100FE0005041A0B0586600401023002037B51A4D7C
:100FF00000F06CFC02236B71184B288119681848AB
:10100000012201F01BFA00230193164B16490093AD
:101010001648174B4FF4805201F066FE154B1978B5
:1010200011B1124801F088FE01F06AFB0446FFF797
:10103000E3FB4FF4C873B0FBF3F202FB130304F5B8
:10104000167010FA83F00C4B186003F047F808B1E3
:101050000F232B8103B030BD8C23002010230020F0
:10106000D8330020090B00089C230020A433002063
:101070000D0C000898230020A03300202DE9F04F2C
:101080002DED028B0FF23829D9E90089834C93B0FA
:101090000BAE9FED7E8BFFF7F1FC814FDFF828A2AE
:1010A00000230A93ADF834300B9373604FF0000BBC
:1010B0005B468DED008B01250DF11D0207A9384619
:1010C0008DF81C508DF81DB001F068F99DF81C30AA
:1010D000002B40F0A580204601F036FE0646002891
:1010E00045D1704F01F00CFB3B6898423FD301F0B3
:1010F00007FB8246FFF780FB4FF4C873B0FBF3F2A7
:1011000002FB13030AF5167010FA83F03860664F7D
:1011100097F800B0CBF1100ABBF1000F14BF3346B3
:101120002B465FFA8AFA0EA88DF82830FFF77CFB71
:10113000BAF1060F28BF4FF0060A0EAB03EB0B0106
:1011400052460DF1290000F03DF90AAB0393182334
:1011500002930AF10102554BD2B2CDE90053049239
:1011600020464CA3D3E9002301F034FE3E7001F089
:10117000C7FA4F4A4F4D1368C31AB3F57A7F2ED37F
:10118000106001F0BFFA02460B46204601F0BAFE9D
:10119000204601F0D9FD10B32B7A474E002B14BF27
:1011A00003230223737101F0ABFA0EAF4FF47A738D
:1011B0000122B0FBF3F039463060304600F006FA09
:1011C000182302933D4B019380B240F25513CDE9B1
:1011D0000370009342464B46204601F0FBFD2B7AFC
:1011E00093B101F08DFA002607464FF48A7A95F8FC
:1011F000D900304400F003000AFB005393F8E820C4
:1012000092B30136042EF2D1C82002F0F3FB2B7A00
:10121000002B7FF43DAF13B0BDEC028BBDE8F08F27
:10122000DAF8143083F48053CAF814305946102287
:101230000EA800F0D9F80DF11E0308AA0AA9384635
:1012400000F028FE96E803000FAB83E803009DF84A
:1012500034308DF844300A9B0E930EA9DDE9082343
:10126000204602F023F821E7D3F8E02042B12B68B2
:10127000FA2B38BFFA23BA1A0533B2EB430FC0D3A7
:10128000FFF7ACFB0028BCD1BEE700BF00000000A8
:1012900000000000401DA12026812A0BA43300205D
:1012A000D8330020A03300209D3300209C33002041
:1012B000D8490020A84400208C230020DC490020CD
:1012C000F1C6A7C1D068080F0004024008B5054860
:1012D00000F07AFEBDE80840034A0449002003F00C
:1012E000C7BC00BFD8330020184A0020D50B000827
:1012F0007047000070B502F041FD094E094D308085
:10130000002428683388834208D902F031FD2B6815
:1013100004440133B4F5803F2B60F2D370BD00BFAD
:101320000C4A0020E049002002F0D8BD00F1006026
:10133000920000F5803002F067BD0000054B1A688E
:10134000054B1B889B1A834202D9104402F010BD42
:1013500000207047E04900200C4A0020024B1B6827
:10136000184402F00DBD00BFE0490020024B1B688D
:10137000184402F01DBD00BFE0490020064991F865
:10138000243033B10023086A81F824300822FFF7A3
:10139000CDBF0120704700BFE4490020022802BFF2
:1013A000024B4FF480529A61704700BF0004024024
:1013B000022802BF024B4FF080529A61704700BF73
:1013C0000004024010B50023934203D0CC5CC45407
:1013D0000133F9E710BD000003460246D01A12F9A6
:1013E000011B0029FAD1704702440346934202D000
:1013F00003F8011BFAE770472DE9F8431F4D144627
:1014000095F824200746884652BBDFF870909CB3BD
:1014100095F824302BB92022FF2148462F62FFF790
:10142000E3FF95F82400C0F10802A24228BF22463B
:10143000D6B24146920005EB8000FFF7C3FF95F856
:101440002430A41B1E44F6B2082E17449044E4B284
:1014500085F82460DBD1FFF791FF0028D7D108E0A1
:101460002B6A03EB82038342CFD0FFF787FF00286C
:10147000CBD10020BDE8F8830120FBE7E449002040
:101480002DE9F0470D46044600219046284640F2DB
:101490007912FFF7A9FF234620220021284601F0F8
:1014A000A7FE231D02222021284601F0A1FE631D74
:1014B00003222221284601F09BFEA31D03222521A1
:1014C000284601F095FE04F1080310222821284641
:1014D00001F08EFE04F1100308223821284601F0A5
:1014E00087FE04F1110308224021284601F080FE06
:1014F00004F1120308224821284601F079FE04F184
:10150000140320225021284601F072FE04F1180332
:1015100040227021284601F06BFE04F120030822CE
:10152000B021284601F064FE04F121030822B8210D
:10153000284601F05DFE04F12207C0263B463146F5
:1015400008222846083601F053FEB6F5A07F07F1C1
:101550000107F3D104F1320308223146284601F095
:1015600047FE002704F1330A94F832304FEAC709E6
:101570009F4209F5A47615D3B8F1000F08D1314682
:1015800004F599730722284601F032FE09F24F163E
:10159000274694F832213B1B93420CD3F01DC00820
:1015A000BDE8F0870AEB070308223146284601F020
:1015B0001FFE0137D8E707F23313314608222846C9
:1015C00001F016FE08360137E3E7000013B50446C4
:1015D0000846002101602346C0F803102022019034
:1015E00001F006FE0198231D0222202101F000FED9
:1015F0000198631D0322222101F0FAFD0198A31D29
:101600000322252101F0F4FD019804F108031022C2
:10161000282101F0EDFD072002B010BDF7B5002331
:10162000047F00910E4607221946054601F0A4FCEE
:10163000731C0093012200230721284601F09CFC23
:10164000C4B9B31C0093052223460821284601F0A3
:1016500093FC0D243746B278BB1B934211D32B7FEA
:10166000A88A0734E408BBB9844294BF0020012053
:1016700003B0F0BDAB8ADB00083BDB08B370082485
:10168000E8E7FB1C0093214600230822284601F0CE
:1016900073FC08340137DEE7201A18BF0120E7E7A2
:1016A000F7B50023047F00910E460822194605462F
:1016B00001F062FC731CC4B9082200931146234652
:1016C000284601F059FC1024012372785F1C013B6D
:1016D000934211D32B7FA88A0734E408BBB9844214
:1016E00094BF0020012003B0F0BDAB8ADB00083BB3
:1016F000DB0873700824E7E7F31900932146002301
:101700000822284601F038FC08343B46DDE7201A61
:1017100018BF0120E7E70000F8B50E46054614465D
:10172000002181223046FFF75FFE2B460822002170
:10173000304601F05DFD7CB96B1C07220821304664
:1017400001F056FD0F2401236A785F1C013B934290
:1017500004D3E01DC008F8BD0824F4E7EB192146C6
:101760000822304601F044FD08343B46ECE7000017
:10177000F8B50E46054614460021CE223046FFF746
:1017800033FE2B4628220021304601F031FD7CB982
:1017900005F1080308222821304601F029FD3024F4
:1017A0002F462A7A7B1B934204D3E01DC008F8BD64
:1017B0002824F5E707F1090321460822304601F005
:1017C00017FD08340137ECE7F7B5047F00910E46AA
:1017D000012310220021054601F0CEFBC4B9B31C41
:1017E0000093092223461021284601F0C5FB192445
:1017F00037467288BB1B9A4211D82B7FA88A0734C0
:10180000E408BBB9844294BF0020012003B0F0BDBE
:10181000AB8ADB00103BDB0873801024E8E73B1D3C
:101820000093214600230822284601F0A5FB083436
:101830000137DEE7201A18BF0120E7E730B5094D70
:101840000A4491420DD011F8013B5840082340F35F
:101850000004013B2C4013F0FF0384EA5000F6D152
:10186000EFE730BD2083B8EDF7B54FF0FF33DFF879
:1018700054C0DFF854E000EB81011A4688421CD0C6
:1018800050F8044B019401AF042417F8015B82EA7D
:1018900005620825DB18164605F1FF355241002E7A
:1018A000BCBF83EA0C0382EA0E0215F0FF05F1D1FA
:1018B000013C14F0FF04E8D1E0E7D843D14303B082
:1018C000F0BD00BF9336EAA9EBE1F042F7B5384A24
:1018D000106851686B4603C36A4636493648082388
:1018E00003F026FA0446002833D10A25334A10684B
:1018F00051686B4603C36A4631492F48082303F0F9
:1019000017FA0446002849D00369B3F5E02F45D8FB
:10191000B0F8661040F2E93291423FD1294A0244C0
:1019200002F15C018B4239D35C3B234900209E1AB3
:10193000FFF784FF3246074604F164010020FFF7F9
:101940007DFFA3689F4229D1E368984208BF002524
:1019500024E00369B3F5E02F27D8418B40F2E93248
:10196000914220D1174A024402F110018B4218D350
:10197000103B114900209D1AFFF760FF2A460646DA
:1019800004F118010020FFF759FFA3689E4202D11D
:10199000E368984201D00D25A8E70025284603B04A
:1019A000F0BD1025A2E70C25A0E70B259EE700BFA0
:1019B000244E0008DCFF0600000001082D4E000840
:1019C00090FF06000800FFF710B5037C044613B92A
:1019D000006803F095F9204610BD00000023BFF316
:1019E0005B8FC360BFF35B8FBFF35B8F8360BFF31D
:1019F0005B8F7047BFF35B8F0068BFF35B8F7047EF
:101A000070B505460C30FFF7F5FF05F108060446F2
:101A10003046FFF7EFFFA04206D930466D68FFF76A
:101A2000E9FF2544281A70BD3046FFF7E3FF201A6E
:101A3000F9E7000070B50546406898B105F1080067
:101A4000FFF7D8FF05F10C0604463046FFF7D2FF3A
:101A50008442304694BF6D680025FFF7CBFF013C00
:101A60002C44201A70BD000038B50C460546FFF71F
:101A7000C7FFA04210D305F10800FFF7BBFF0444E5
:101A80006868B4FBF0F100FB1144BFF35B8F0120E9
:101A9000AC60BFF35B8F38BD0020FCE72DE9F0415F
:101AA000144607460D46FFF7C5FF844228BF04468B
:101AB000D4B1B84658F80C6B4046FFF79BFF304452
:101AC000286040467E68FFF795FF331A9C4203D892
:101AD0006C600120BDE8F0816B60A41B3B68AB60CB
:101AE0002044E8600220F5E72046F3E738B50C46CD
:101AF0000546FFF79FFFA04210D305F10C00FFF74A
:101B000079FF04446868B4FBF0F100FB1144BFF3B3
:101B10005B8F0120EC60BFF35B8F38BD0020FCE7DA
:101B20002DE9FF41884669460746FFF7B7FF6C4637
:101B300006B204EBC6060025B44209D062682068EC
:101B400008EB0501FFF73EFC636808341D44F3E72A
:101B500029463846FFF7CAFF284604B0BDE8F081A1
:101B6000F8B505460C300F46FFF744FF05F10806AF
:101B700004463046FFF73EFFA042304688BF6C68FF
:101B8000FFF738FF201A386020B130462C68FFF785
:101B900031FF2044F8BD000073B5144606460D46DB
:101BA000FFF72EFF844228BF04460190DCB101A953
:101BB0003046FFF7D5FF019B33B93268C5E90233E0
:101BC000C5E9002401200CE09C4238BF0194286044
:101BD000019868608442F5D93368AB60241AEC60E0
:101BE000022002B070BD2046FBE700002DE9FF4156
:101BF0000F466946FFF7D0FF6C4600B204EBC00504
:101C00000026AC4209D0D4F8048054F8081BB81957
:101C10004246FFF7D7FB4644F3E7304604B0BDE841
:101C2000F081000038B50546FFF7E0FF04460146A5
:101C30002846FFF719FF204638BD0000302383F304
:101C4000118862B670470000002383F3118862B6E2
:101C50007047000010B4026854681A4623465DF8C5
:101C6000044B184701207047002070470020704740
:101C700070470000002070470E20704700F580502C
:101C800090F8C800C0F340007047000000F5805095
:101C900090F9C90070470000F7B50C68BDF82070D6
:101CA00014F000541E466FD10B7B082B6CD8FFF745
:101CB000C5FF4569AB685B010CD4AB681B0108D458
:101CC000AC6814F080545DD1FFF7BEFF204603B02E
:101CD000F0BD01240B6804F1180C002BB8BFDB0029
:101CE0004FEA0C1CB4BF43F004035B0545F80C300D
:101CF0000B680FFA84FC13F0804F18BF05EB0C1E25
:101D000005EB0C1C1EBFDEF8803143F00203CEF859
:101D100080310B7BCCF8843105EB04158B68C5F85A
:101D20008C314B68C5F88831DCF8803143F0010311
:101D3000CCF8803100EB441541F268031D4403EBFD
:101D400044130344C5E9002608330D4601F10C0C89
:101D500055F804EB43F804EB6545F9D184342D883C
:101D60001D8000EB441407F00303257925F00B05D3
:101D70002B432371FFF768FF0097334600F0E2FC26
:101D80000120A4E70224A5E74FF0FF309FE7000001
:101D900013B500F580540191E06DFFF74BFE1F284D
:101DA0000AD90199E06D2022FFF7BAFEA0F12003C5
:101DB0005842584102B010BD0020FBE708B500F5BD
:101DC0008050FFF73BFFC06DFFF708FEBDE80840FD
:101DD000FFF73ABF00220260828142608260704752
:101DE00010B500220023C0E900230023044603812C
:101DF0000C30FFF7EFFF204610BD0000F0B50546A0
:101E000000F580500C4690F8C83013F0040FC3F36F
:101E1000800108BF114661F3820304F1840680F853
:101E2000C83005EB461389B01B79D8072ED57AB395
:101E300019072DD46846FFF7D3FF05EB441303F5CC
:101E4000835303F1180703AA10331868596814461E
:101E500003C40833BB422246F7D1186820609B8830
:101E6000A380DDE90E23CDE900230123ADF808307E
:101E70002B686946DB6B2846984705EB46152B799E
:101E80001A075CBF43F008032B7101E0002AF4D16C
:101E900009B0F0BD2DE9F047074688B007F580543A
:101EA00068469A468846FFF7C9FE9146FFF798FFB5
:101EB000E06DFFF7A5FD1F2829D9E06D20226946B6
:101EC000FFF7B0FE202822D103AD444605AB2E46D5
:101ED00003CE9E4220606160354604F10804F6D1CD
:101EE00030682060B388A380DDE90023C9E90023BE
:101EF000BDF80830AAF80030FFF7A6FE4A46534660
:101F00004146384608B0BDE8F04700F009BCFFF78D
:101F10009BFE002008B0BDE8F08700002DE9F84FD7
:101F20000023C0E90133254B044640F8183B0F4617
:101F3000FFF750FF04F12800FFF752FF04F14808B3
:101F400004F582554646083530462036FFF748FFEF
:101F5000AE42F9D104F580554FF480534FF000099B
:101F6000C5E91339C5F848800123EE6504F58758A3
:101F700004F58456C5F8549085F8583085F86030DB
:101F8000083608F108084FF0000A4FF0000B46E948
:101F900008ABA6F11800FFF71DFF203646F8289C75
:101FA0004645F4D185F8C97017B1054800F0A2FB89
:101FB000044B63612046BDE8F88F00BF604E000807
:101FC000384E00080064004010B5044B19780446F0
:101FD0004A1C1A70FFF7A2FF204610BD144A0020C9
:101FE0002DE9F047002950D0294B2A4FB7FBF1F5D6
:101FF00099428CBF0A231123581EB5FBF3FC03FB47
:102000001C53C4B22BB102280346F5D80020BDE80A
:10201000F0870CF1FF36B6F5806FF7D2C4EBC40E33
:102020000EF103034FEAE309C3F3C703A4EB03086C
:1020300009F1010A4FF47A755FFA88F009FB05553A
:102040005AFA88F8B5FBF8F5B5F5617FC1BF0EF116
:10205000FF33C3F3C703E01AC0B25C1C50FA84F428
:102060000CFB04F4B7FBF4F4A142CFD1013BDBB28B
:102070000F2BCBD80138C0B20728C7D80021107168
:1020800016809170D3700120C1E70846BFE700BFFA
:102090003F420F0040787D0170B505460E464FF473
:1020A0007A746B695B6803F00103B34207D04FF4A5
:1020B0007A7001F09FFC013CF3D1204670BD0120F5
:1020C000FCE7000030B54269936913F0700F16D039
:1020D00000230B4C936103F1840200EB421211794F
:1020E0004D0709D5890707D5416954F823508D60FC
:1020F000117941F0040111710133032BEBD130BD93
:102100004C4E000873B51D46436916469A68D207BF
:10211000044609D59A6801219960C2F34002CDE9CD
:1021200000650021FFF76AFE63699A68D1050BD547
:102130009A684FF480719960C2F34022CDE900653E
:1021400001212046FFF75AFE63699A68D2030BD536
:102150009A684FF480319960C2F34042CDE900653E
:1021600002212046FFF74AFE204602B0BDE870403B
:10217000FFF7A8BFF8B50446466900296CD106F1FF
:102180000C07386880076AD006EB01153868D5F867
:10219000B00110F0040FD5F8B0011ABFC00840F02C
:1021A0000040400DA061D5F8B0C11CF0020F1CBF6B
:1021B00040F08040A061D5F8B40106EB011100F0B9
:1021C0000F0084F82400D1F8B8012077D1F8B801C5
:1021D000000A6077D1F8B801000CA077D1F8B801F7
:1021E000000EE077D1F8BC0184F82000D1F8BC01E2
:1021F000000A84F82100D1F8BC01000C84F8220008
:10220000D1F8BC11090E84F823103821396004F18B
:10221000340004F1180104F1240551F8046B40F86E
:10222000046BA942F9D109880180C4E90A23214637
:102230000023238651F8283B2046DB6B984704F5A2
:102240008052204692F8C83043F0040382F8C83028
:10225000BDE8F840FFF736BF06F1100791E7F8BD7B
:1022600010B5044600F04EFA02460B4652EA03014E
:1022700002D0013A63F100030449086820B1214605
:10228000BDE81040FFF776BF10BD00BF104A002028
:10229000F8B500F583511E46FFF7D0FCDFF844C0C7
:1022A0000831002404F1840500EB45152B795F0704
:1022B0000ED4DB060CD5D1E900739742B34107D2A7
:1022C00043695CF824709F602B7943F004032B7101
:1022D0000134032C01F12001E4D1BDE8F840FFF7FF
:1022E000B3BC00BF4C4E000808B5FFF7A7FCFFF7D2
:1022F000E9FEBDE80840FFF7A7BC0000F8B5436958
:102300000546986800F0E050B0F1E05F0F461FD03E
:10231000E8B1FFF793FC05F583541034002606F16D
:10232000840305EB43131B791A0706D50136032EE8
:1023300004F12004F3D1012007E05B07F6D4214625
:10234000384600F039FA0028F0D1FFF77DFCF8BDDF
:102350000120FCE700F5805008B5FFF76FFCC06D69
:10236000FFF74EFBFFF770FC43090CBF0120002074
:1023700008BD0000F8B51D46002313700F46064641
:102380001446FFF7E7FF80F00100387025B12946B9
:102390003046FFF7B3FF2070F8BD00002DE9B841CB
:1023A0000C4615461F46804600F0ACF90B462178D6
:1023B000024609B9287850B14046FFF769FFFFF798
:1023C00093FF3B462A462146FFF7D4FF0120BDE894
:1023D000B881000010B5FFF731FC174B1A6C42F0C2
:1023E00000721A641A6A42F000721A621A6A00F5E0
:1023F000805422F000721A62FFF726FC94F8C8306D
:10240000DB0718D4B9B103211320FFF717FC01F043
:10241000C7F90321142001F0C3F90321152001F0AD
:10242000BFF994F8C83043F0010384F8C830BDE820
:102430001040FFF709BC10BD003802402DE9F047FD
:1024400000F5805588B095F8C930012B04468846C0
:1024500016467FD8804F57F823200AB947F8230043
:10246000D7F800A0C4F80C802674BAF1000F63D02E
:1024700095F8C930012B6FD001212046FFF7AAFF44
:10248000FFF7DCFB6269136823F0020313606269E3
:10249000136843F001031360636900275F61012142
:1024A0002046FFF7D1FBFFF7F7FD002800F09580ED
:1024B000E86DFFF793FA04F58359BA4609F1080964
:1024C000202200216846FEF78FFF02A8FFF782FC5A
:1024D000CDF818A06A4609EB07030DF1180E9446D3
:1024E000BCE80300F44518605960624603F1080334
:1024F000F5D1DCF80000186020379CF804201A7130
:10250000602FDDD195F8C8306FF38203002785F87E
:10251000C8306A4641462046ADF80070ADF80270FA
:102520008DF80470FFF75CFD636948BB4FF400420F
:102530001A6008B0BDE8F08741F2D00002F0A0FBBD
:10254000814610B15146FFF7E9FCC7F80090B9F198
:10255000000F8DD10020ECE7386803681B6B9847AB
:102560000146002888D13868FFF734FF38680368CF
:1025700032465B684146984700287FF47DAFE9E723
:1025800061221A609DF802309DF803201B06120498
:1025900002F4702203F040731343BDF80020C2F32D
:1025A000090213439DF804201205022E02F4E002F2
:1025B0000CBF4FF000410021134362690B43D3610C
:1025C000636913225A616269136823F0010313607F
:1025D00039462046FFF760FD08B96369A6E795F81C
:1025E000C93093BB6169D1F8002242F00102C1F801
:1025F00000226169D1F8002222F47C5222F00E02FE
:10260000C1F800226169D1F8002242F46062C1F889
:1026100000226269C2F814326269C2F80432626947
:1026200041F6FF71C2F80C126269C2F84032626969
:10263000C2F8443263690122C3F81C226269D2F8ED
:10264000003223F00103C2F8003295F8C83043F09D
:10265000020385F8C8306CE7104A002008B500F086
:1026600051F850EA0103024602D0421E61F1000116
:10267000044B186810B10B46FFF744FDBDE8084055
:1026800001F064B8104A002008B50020FFF7E8FD0B
:10269000BDE8084001F05AB808B50120FFF7E0FD99
:1026A000BDE8084001F052B800B59BB0EFF30981D6
:1026B00068226846FEF786FEEFF30583014B9B6BAD
:1026C000FEE700BF00ED00E008B5FFF7EDFF0000FA
:1026D00000B59BB0EFF3098168226846FEF772FEF1
:1026E000EFF30583014B5B6BFEE700BF00ED00E0FD
:1026F000FEE700000FB408B5029801F011F9FEE7FB
:1027000001F038BC01F010BC13B56C4684E806003B
:10271000031D94E8030083E80500012002B010BD0A
:1027200073B58568019155B11B885B0707D4D0E963
:1027300000369B6B9847019AC1B23046A8470120EA
:1027400002B070BDF0B5866889B005460C465EB132
:10275000BDF838305B070AD4D0E900379B6B984747
:102760002246C1B23846B047012009B0F0BD002270
:102770000023CDE900230023ADF808300A4603AB5F
:1027800001F10806106851681C4603C40832B242C1
:102790002346F7D1106820609288A280FFF7B2FF2D
:1027A0000423ADF808302B68CDE90001DB6B6946E6
:1027B00028469847D8E7000030B503680968DD0F60
:1027C000B5EBD17F23F0604421F060424FEAD17035
:1027D0000BD0002BB8BFA40C0029B8BF920C9442B8
:1027E00002D034BF0120002030BD944205D1C1F396
:1027F0008070C3F380738342F6D194422CBF0020D3
:102800000120F1E72DE9F041456A15B94162BDE8C3
:10281000F0814B6823F06047C3F38A464FEAD37ECA
:10282000C3F3807816EA230638BF3E46AC462B46F3
:102830005A68BEEBD27F22F060440AD0002A18DA30
:10284000A40CB44217D19D420FD10D60DEE71346B0
:10285000EEE7A74207D102F08044C2F380724245FE
:102860000BD054B1EFE708D2EDE7CCF800100B60C5
:10287000CDE7B44201D0B442E5D81A689C46002A9C
:10288000E5D11960C3E700002DE9F047089D01F08C
:1028900007044FEAD508224405F0070500EBD100F4
:1028A0004FF47F49944201D1BDE8F08704F0070757
:1028B00005F0070A57453E4638BF5646C6F108069A
:1028C000111B8E4228BF0E46E10808EBD50E415C75
:1028D00013F80EC0B94029FA06F721FA0AF1FFB23F
:1028E0008CEA010147FA0AF739408CEA010C03F837
:1028F0000EC034443544D5E780EA0120082341F274
:10290000210201B24000002980B203F1FF33B8BFB9
:10291000504013F0FF03F4D17047000038B50C4667
:102920008D18A54200D138BD14F8011BFFF7E4FF54
:10293000F7E7000042684AB1136843604389818920
:1029400001339BB29942438138BF8381104670475F
:1029500070B588B0202204460D4668460021FEF777
:1029600043FD20460495FFF7E5FF024658B16B464C
:10297000054608AE1C4603CCB44228606960234675
:1029800005F10805F6D1104608B070BD082817D922
:1029900009280CD00A280CD00B280CD00C280CD0FD
:1029A0000D280CD00E2814BF4020302070470C207A
:1029B000704710207047142070471820704720205F
:1029C00070470000082817D90C280CD910280CD9FA
:1029D00014280CD918280CD920280CD930288CBFE1
:1029E0000F200E207047092070470A2070470B20E7
:1029F00070470C2070470D20704700002DE9F84308
:102A0000078C072F04461ED9D0E9029800254FF6FF
:102A1000FF73C5F12006A5F1200029FA05F108FA97
:102A200006F628FA00F031430143C9B21846FFF711
:102A300063FF0835402D0346EBD1E1693A46BDE816
:102A4000F843FFF76BBF4FF6FF70BDE8F883000057
:102A500010B54B6823B9CA8A63F30902CA8210BD54
:102A600004691A681C600361C38A013BC3824A601F
:102A7000EFE700002DE9F84F1D46CB8A0F46C3F360
:102A800009010529814692460B4630D00020AAB2A2
:102A900007F11A049EB2042E1FFA80F80FD8904551
:102AA00003F1010306D3FB8A0A4462F30903FB82A4
:102AB00001201AE01AF80060E6540130EAE7904578
:102AC000F1D2A1F1050B1C237C68BBFBF3F203FBE5
:102AD00012BB1FFA8BF6002C45D14846FFF72AFFA0
:102AE000044638B978606FF00200BDE8F88F4FF007
:102AF0000008E6E7002606607860ADB24FF0000BF4
:102B0000454510D90AEB0803221D13F8011B915506
:102B1000B1B208F101081B291FFA88F82BD04545EE
:102B200006F10106F1D8FB8AC3F30902154465F3E7
:102B30000903BCE7013292B21C462368002BF9D18D
:102B40006B1F0B441C21B3FBF1F301339BB29A4280
:102B5000D3D2BBF1000FD0D14846FFF7EBFE20B92E
:102B6000C4F800B0BFE70122E7E7C0F800B05E4656
:102B700020600446C1E74545D5D94846FFF7DAFE4F
:102B800008B92060AFE7C0F800B000262060044616
:102B9000B6E700002DE9F04F2DED028B1C4683B007
:102BA0005B69019207468846002B00F09A80238CCF
:102BB0002BB1E269002A00F09480072B35D807F189
:102BC0000C00FFF7B7FE054638B96FF0020528463E
:102BD00003B0BDEC028BBDE8F08F14220021FEF79C
:102BE00003FC228CE16905F10800FEF7EBFB208C69
:102BF000013080B2FFF7E6FEFFF7C8FE013880B271
:102C00002084013028746369228C1B782A4403F0E5
:102C10001F0363F03F0348F00041137238466960B8
:102C20002946FFF7EFFD0125D1E700F10C034FF036
:102C3000000908EE103A4FF0800A4E464D4618EE55
:102C4000100AFFF777FE83460028BED01422002129
:102C5000FEF7CAFB002E3AD1019BABF808300222E6
:102C60000BF1080E1FFA82FC0CF10100BCF1060FFB
:102C7000218C80B201D88E422BD3FFF7A3FEFFF741
:102C800085FE62691278013802F01F028E4208BF89
:102C90004FF0400A42EA49121BFA80F14AEA020A5E
:102CA000013048F0004281F808A08BF81000CBF802
:102CB000042059463846FFF7A5FD238C0135B34261
:102CC0002DB289F001094FF0000AB8D17FE7002248
:102CD000C6E7E169895D0EF802100136B6B201322D
:102CE000C0E76FF0010572E7F8B515460E463022D1
:102CF000002104461F46FEF777FB069B6360B5F58F
:102D0000001F079BA76034BF6A094FF6FF72A362DA
:102D100097B2E66104F1100000239A4206D800231E
:102D20000360A782E3822383E360F8BD066001337A
:102D300030462036F1E7000003781BB94BB2002B78
:102D4000C8BF01707047000000787047F8B50C46A6
:102D5000C969074611B9238C002B37D1257E1F2D59
:102D600034D8387828BB228C072A2CD8268A36F00B
:102D700003032BD14FF6FF70FFF7D0FD20F00100C9
:102D80003102400441EA0561400C41EA40254FF61A
:102D9000FF72234629463846FFF7FCFE002807DD70
:102DA000626913780133DBB21F2B88BF00231370D5
:102DB000F8BD218A2D0645EA012505432046FFF787
:102DC0001DFE0246E5E76FF00300F1E76FF001003A
:102DD000EEE7000070B58AB00446164600212822AE
:102DE00068461D46FEF700FBBDF83830ADF81030E0
:102DF0000F9B05939DF840308DF81830119B079379
:102E00006946BDF84830ADF820302046CDE902656E
:102E1000FFF79CFF0AB070BD2DE9F041D36905466C
:102E20000C4616460BB9138C5BBB377E1F2F28D878
:102E300095F80080B8F1000F26D03046FFF7DEFD90
:102E40003378210241EAC33141EA0801338A41EA79
:102E5000076141EA03410246334641F080012846BA
:102E6000FFF798FE00280ADD3378012B07D172693D
:102E700013780133DBB21F2B88BF00231370BDE82A
:102E8000F0816FF00100FAE76FF00300F7E7000050
:102E9000F0B58BB004460D4617460021282268463F
:102EA0001E46FEF7A1FA9DF84C305A1E534253417C
:102EB0008DF800309DF84030ADF81030119B05932F
:102EC0009DF848308DF81830149B07936A46BDF87A
:102ED0005430ADF8203029462046CDE90276FFF780
:102EE0009BFF0BB0F0BD0000406A00B1043070479A
:102EF000436A1A68426202691A600361C38A013B2D
:102F0000C38270472DE9F041D0F82080194E144655
:102F10001D464146002709B9BDE8F081D1E90223E9
:102F2000A21A65EB0303964277EB03031ED2036AF2
:102F30008B420DD1FFF78CFD036A1B6803620369A6
:102F40000B60C38A0161016A013BC3828846E2E7E4
:102F5000FFF77EFD0B68C8F8003003690B60C38A79
:102F60000161013BC382D8F80010D4E788460968A4
:102F7000D1E700BF80841E002DE9F04F8BB00D46D5
:102F8000DDF8509014469B468046002800F01981D9
:102F9000B9F1000F00F01581531E3F2B00F2118193
:102FA000012A03D1BBF1000F40F00B810023CDE9D2
:102FB0000833B8F81430B5EBC30F4FEAC30703D397
:102FC00000200BB0BDE8F08F2B199F42D8F80C30D1
:102FD0003ABF7F1BFFB227461BB9D8F81030002B31
:102FE0007AD0272D4ED8C5F12806B7424FF00003FE
:102FF0002CBFF6B23E4600932946D8F8080008AB2D
:103000003246FFF741FCA7EB060A35445FFA8AFA1D
:10301000B8F8143003F10053053BDB000493D8F8F3
:103020000C3003932821039B13B1BAF1000F2CD16C
:10303000D8F8100040B1BAF1000F05D0009608ABE7
:103040005246691AFFF720FC38B2002FB8D0660745
:103050000AD00AAB03EBD401624211F8083C02F03B
:103060000702134101F8083C082C3CD9102C40F20F
:10307000B580202C40F2B780BBF1000F00F09C809F
:10308000082334E0BA460026C2E7049BE02B28BFA1
:10309000E02306930B44AB42059314D95A1B0398C3
:1030A0000096924534BF5246D2B2691A08AB04303A
:1030B0000792FFF7E9FB079A1644AAEB020A1544A8
:1030C000F6B25FFA8AFA049B069A05999B1A049352
:1030D000039B1B680393A6E70093D8F8080008AB8E
:1030E0003A462946AEE7BBF1000F13D00123B4EBFB
:1030F000C30F6CD0082C12D89DF82030621E23FA22
:1031000002F2D50706D54FF0FF3202FA04F423434A
:103110008DF820309DF8203089F8003051E7102CD0
:1031200012D8BDF82030621E23FA02F2D10706D56C
:103130004FF0FF3202FA04F42343ADF82030BDF81B
:103140002030A9F800303CE7202C0FD80899631EE6
:1031500021FA03F3DA0705D54FF0FF3202FA04F43F
:103160000C430894089BC9F800302AE7402C2BD068
:10317000DDE90865611EC4F12102A4F1210326FAEC
:1031800001F105FA02F225FA03F311431943CB07C3
:1031900012D50122A4F12003C4F1200102FA03F3A5
:1031A00022FA01F1A240524243EA010363EB4303D6
:1031B00032432B43CDE90823DDE90823C9E9002385
:1031C000FFE66FF00100FCE66FF00800F9E6082C5E
:1031D000A0D9102CB3D9202CEED8C3E7BBF1000F37
:1031E000ADD0022383E7BBF1000FBBD004237EE701
:1031F00030B5012A144638BF0124402C85B028BFC1
:1032000040240025012ACDE9025518D81B788DF8F5
:10321000083063070AD004AB03EBD405624215F80B
:10322000083C02F00702934005F8083C0091034671
:103230002246002102A8FFF727FB05B030BD082A6F
:10324000E4D9102A03D81B88ADF80830E1E7202A1A
:103250008DBFD3E900231B680293CDE90223D8E791
:1032600010B5CB681BB98B600B618B8210BD0469F4
:103270001A681C600361C38A013BC382CA60F0E71D
:1032800003064CBFC0F3C0300220704708B50246A9
:10329000FFF7F6FF022806D15306C2F30F2001D133
:1032A00000F0030008BDC2F30740FBE72DE9F04F33
:1032B00093B0CDE903230A6804461046FFF7E0FF08
:1032C000022814BFC2F306260026002A0D468246B5
:1032D00080F2F28112F0C04940F0EE81097B0029B2
:1032E00000F0EA81022803D02378B34240F0E7815E
:1032F000C2F304630693104602F07F030593FFF7C1
:10330000C5FF059B29444FEA834848EA0A4848EA32
:103310004668CE7800230022CDE90823F3098346CE
:1033200048EA0008029367D0059B0093024667684D
:10333000534608A92046B847002800F0C381276AF1
:103340004FB9414604F10C00FFF702FB074690B964
:103350006FF0020054E03B6998450DD03F68002FA4
:10336000F9D1414604F10C00FFF7F2FA07460028B4
:10337000EED0236A3B60276297F817C006F01F085B
:10338000CCF3840CACEB08001FFA80FE0028B8BF19
:103390000EF12000A8EB0C031FFA83FED7E90221EF
:1033A000B8BF00B2002B0793BEBF0EF120031BB2C3
:1033B000079352EA010338D0039BDFF824E39A1AFB
:1033C000049B4FF0000C63EB010196457CEB01037D
:1033D0002BD36B7B97F81AE0734519D1029B002B16
:1033E00078D0012821DC7868F8B9DFF8F0C294457C
:1033F00070EB010316D337E0276A27B96FF00C0092
:1034000013B0BDE8F08F3B699845B5D03F68F4E74D
:10341000B24890427CEB010301D30020F0E7029B0D
:10342000002BFAD0079B0F2B17DCFA7DB30002F0BC
:10343000030203F07C031343FB7539462046FFF774
:1034400007FB6B7BBB76029B3BB9FB7DC3F384021E
:10345000013262F38603FB75D0E76A7BBB7E9A423A
:10346000DBD1029B002B35D0B309022B32D0039B5A
:10347000BB60049BFB60142200210DA8FDF7B4FF84
:10348000039B0A93049B0B932B1D0C932B7BADF892
:103490003EB0013BDBB2ADF83C30069B8DF84230CC
:1034A000059B8DF8433094F82C308DF840A083F0C4
:1034B00001038DF844308DF84180A3680AA92046A5
:1034C0009847FB7DC3F38403013303F01F039B0282
:1034D000FB82A2E7FB7DC6F34012B2EBD31F40F0A4
:1034E000F480C3F38403434540F0F280029A2B7BBF
:1034F000B609002A4DD0F2075DD4032B40F2EB80D1
:10350000039BBB60049BFB602B7BAE1D033BDBB2CC
:103510003246394604F10C00FFF7ACFA00280CDA09
:1035200039462046FFF794FAFB7DC3F38403013349
:1035300003F01F039B02FB820AE7DDE90884AB88E6
:103540003B834FF6FF73C9F12000A9F1200228FA4E
:1035500009F104FA00F0014324FA02F2114318467B
:10356000C9B2FFF7C9F909F10809B9F1400F0346DB
:10357000E9D1B8822A7B033AD2B23146FFF7CEF9BD
:10358000FB7DB882DA43C2F3C01262F3C713FB7546
:1035900043E786B92E1D013BDBB23246394604F1C2
:1035A0000C00FFF767FA0028BADB2A7BB88A013AD9
:1035B000D2B23146E2E7F98AC1F30901013B04299D
:1035C000DAB25BD8281D002307F11B069A4208D9FE
:1035D00010F801CB06F801C0013101330529DBB237
:1035E000F4D103990A9104990B91934207F11B01BD
:1035F0000C9138BF043379680D9134BF55FA83F3C9
:1036000000230E93FB8AADF83EB0C3F309031A44BE
:10361000069B8DF84230059B8DF8433094F82C3092
:10362000ADF83C2083F001038DF8443000238DF881
:1036300040A08DF841807B602A7BB88A013A291D21
:10364000FFF76CF93B8BB882834203D1A3680AA9C8
:103650002046984720460AA9FFF702FEFB7DBA8A5A
:10366000C3F38403013303F01F039B02FB823B8BF4
:103670009A420CBF00206FF01000C1E67B68002B5F
:10368000AFD0052001E01C3033461E68002EFAD171
:10369000091A081D2E1D184401EB090CBCF11B0F63
:1036A0005FFA89F39DD89A429BD916F8013B00F83E
:1036B000013B09F10109EFE76FF00900A0E66FF0A7
:1036C0000A009DE66FF00B009AE66FF00D0097E69A
:1036D0006FF00E0094E66FF00F0091E640420F008D
:1036E00080841E00EFF3098305494A6B22F0010232
:1036F0004A63683383F30988002383F31188704792
:1037000000EF00E0302080F3118862B60C4B0D4AC8
:10371000D96821F4E0610904090C0A43DA60D3F89E
:10372000FC20094942F08072C3F8FC200A6842F08C
:1037300001020A602022DA7783F82200704700BF76
:1037400000ED00E00003FA05001000E010B53023A2
:1037500083F311880E4B5B6813F4006314D0F1EE11
:10376000103AEFF30984683C4FF08073E361094B32
:10377000DB6B236684F3098800F090F810B1064BE8
:10378000A36110BD054BFBE783F31188F9E700BF88
:1037900000ED00E000EF00E04306000846060008E8
:1037A00000F1604303F561430901C9B283F80013D6
:1037B000012200F01F039A4043099B0003F160437C
:1037C00003F56143C3F880211A6070470023037535
:1037D000826803691B6899689142FBD25A6803604A
:1037E0004260106058607047002303758268036967
:1037F0001B6899689142FBD85A6803604260106068
:103800005860704708B50846302383F311880B7D54
:10381000032B05D0042B0DD02BB983F3118808BDE1
:103820008B6900221A604FF0FF338361FFF7CEFFF0
:103830000023F2E7D1E9003213605A60F3E7000099
:10384000FFF7C4BF054BD9680875186802681A608D
:10385000536001220275D860FCF7DEBE204A0020CA
:1038600030B50C4BDD684B1C87B004460FD02B469F
:10387000094A684600F06CF92046FFF7E3FF009B19
:1038800013B1684600F06EF9A86907B030BDFFF7C4
:10389000D9FFF9E7204A002005380008044B1A68D0
:1038A000DB6890689B68984294BF002001207047B5
:1038B000204A0020084B10B51C68D86822681A609E
:1038C000536001222275DC60FFF78EFF014620461F
:1038D000BDE81040FCF7A0BE204A0020044B1A6847
:1038E000DB6892689B689A4201D9FFF7E3BF704793
:1038F000204A002038B5074C074908480123002515
:103900002370656000F03AFC0223237085F3118870
:1039100038BD00BF884C0020A44E0008204A00207B
:1039200008B572B6044B186500F0ECFA00F0A0FB85
:10393000024B03221A70FEE7204A0020884C002028
:1039400000F046B9EFF3118020B9EFF30583302280
:1039500082F311887047000010B530B9EFF3058489
:10396000C4F3080414B180F3118810BDFFF7B6FF4B
:1039700084F31188F9E700008B60022308618B82D1
:10398000084670478368A3F1840243F8142C026947
:1039900043F8442C426943F8402C094A43F8242C4C
:1039A000C26843F8182C022203F80C2C002203F8FA
:1039B0000B2C044A43F8102CA3F12000704700BFE1
:1039C00031060008204A002008B5FFF7DBFFBDE8FC
:1039D0000840FFF735BF0000024BDB6898610F20FD
:1039E000FFF730BF204A0020302383F31188FFF710
:1039F000F3BF000008B50146302383F31188082087
:103A0000FFF72EFF002383F3118808BD064BDB6808
:103A100039B1426818605A60136043600420FFF7B0
:103A20001FBF4FF0FF307047204A002003689842C4
:103A300006D01A680260506099611846FFF700BF0F
:103A40007047000010B503689C68A2420CD85C68FF
:103A50008A600B604C602160596099688A1A9A608C
:103A60004FF0FF33836010BD1B68121BECE70000B2
:103A70000A2938BF0A2170B504460D460A26601986
:103A800000F076FB00F062FB041BA54203D8751C16
:103A90002E460446F3E70A2E04D9BDE87040012003
:103AA00000F0ACBB70BD0000F8B5144B0D46D961F9
:103AB00003F1100141600A2A1969826038BF0A22A5
:103AC000016048601861A818144600F043FB0A27FB
:103AD00000F03CFB431BA342064606D37C1C28197E
:103AE00000F046FB27463546F2E70A2F04D9BDE829
:103AF000F840012000F082BBF8BD00BF204A002042
:103B0000F8B506460D4600F021FB0F4A134653F860
:103B1000107F9F4206D12A4601463046BDE8F84054
:103B2000FFF7C2BFD169BB68441A2C1928BF2C46C5
:103B3000A34202D92946FFF79BFF2246314603489C
:103B4000BDE8F840FFF77EBF204A0020304A002041
:103B500010B4C0E9032300235DF8044B4361FFF771
:103B6000CFBF000010B5194C236998420DD0D0E9A1
:103B70000032816813605A609A680A449A60002390
:103B800003604FF0FF33A36110BD2346026843F882
:103B9000102F53600022026022699A4203D1BDE8CF
:103BA000104000F0DFBA936881680B44936000F026
:103BB000CDFA2269E1699268441AA242E4D911441B
:103BC000BDE81040091AFFF753BF00BF204A00208C
:103BD0002DE9F047DFF8BC8008F110072C4ED8F82B
:103BE000105000F0B3FAD8F81C40AA68031B9A42A0
:103BF0003ED81444D5E900324FF00009C8F81C4003
:103C000013605A60C5F80090D8F81030B34201D163
:103C100000F0A8FA89F31188D5E9033128469847BE
:103C2000302383F311886B69002BD8D000F08EFA13
:103C30006A69A0EB04094A4582460DD2022000F0D1
:103C4000DDFA0022D8F81030B34208D15146284698
:103C5000BDE8F047FFF728BF121A2244F2E712EB43
:103C6000090938BF4A4629463846FFF7EBFEB5E753
:103C7000D8F81030B34208D01444211AC8F81C00F8
:103C8000A960BDE8F047FFF7F3BEBDE8F08700BFCD
:103C9000304A0020204A002000207047FEE7000044
:103CA000704700004FF0FF3070470000BFF34F8FA8
:103CB000024AD368DB03FCD4704700BF003C0240DB
:103CC00008B5094B1B7873B9FFF7F0FF074B1A696A
:103CD000002ABFBF064A5A6002F188325A601A6849
:103CE00022F480621A6008BD904C0020003C024023
:103CF0002301674508B50B4B1B7893B9FFF7D6FF37
:103D0000094B1A6942F000421A611A6842F4805263
:103D10001A601A6822F480521A601A6842F48062AB
:103D20001A6008BD904C0020003C02400728F0B506
:103D300016D80C4C0C4923787BB90C4D0E46082341
:103D40004FF0006255F8047B46F8042B013B13F05A
:103D5000FF033A44F6D10123237051F82000F0BD4F
:103D60000020FCE7B44C0020944C0020B04E00082A
:103D7000014B53F820007047B04E000808207047F0
:103D8000072810B5044601D9002010BDFFF7CEFF6B
:103D9000064B53F824301844C21A0BB90120F4E73B
:103DA00012680132F0D1043BF6E700BFB04E0008C4
:103DB000072810B5044621D8FFF778FFFFF780FFEA
:103DC0000F4AF323D360C300DBB243F4007343F024
:103DD00002031361136943F480331361FFF766FF35
:103DE000FFF7A4FF074B53F8241000F03DF9FFF74D
:103DF00081FF2046BDE81040FFF7C2BF002010BD84
:103E0000003C0240B04E0008F8B512F00103144621
:103E100042D185182E4A954257D82E4B1B6813F075
:103E2000010352D02C4DFFF74BFFF323EB60FFF75C
:103E30003DFF40F20127032C15D824F00104661839
:103E4000254C401A40F20117B142236900EB0105ED
:103E500024D123F001032361FFF74CFF0120F8BDBB
:103E6000043C0430E7E78307E7D12B6923F4407370
:103E70002B612B693B432B6151F8046B0660BFF348
:103E80004F8FFFF713FF03689E42E9D02B6923F0A1
:103E900001032B61FFF72EFF0020E0E723F44073BE
:103EA000236123693B4323610B882B80BFF34F8F32
:103EB000FFF7FCFE2D8831F8023BADB2AB42C3D018
:103EC000236923F001032361E4E71846C7E700BF35
:103ED0000000080800380240003C0240084908B5CC
:103EE0000B7828B11BB9FFF7EBFE01230B7008BD5F
:103EF000002BFCD0BDE808400870FFF7FBBE00BFF8
:103F0000904C00204FF480214FF0005000F0AEB8EC
:103F10000846114600F0D6BE012000F0D3BE0000D6
:103F2000084600F0EDBE000070B582B0FFF70AFD54
:103F30000E4E054600F00AF93268904237BF0C4A2F
:103F40000B49516814682EBFD1E90041013151601D
:103F50000419034641F10001284601913360FFF73F
:103F6000FBFC0199204602B070BD00BFB84C002098
:103F7000C04C002070B582B0FFF7E4FC104E05463F
:103F800000F0E4F83268904237BF0E4A0D4951689C
:103F900014682EBFD1E9004101315160041941F18B
:103FA00000010346284601913360FFF7D5FC0199D3
:103FB0004FF47A7200232046FCF71AF902B070BD64
:103FC000B84C0020C04C002010B50244064BD2B2C1
:103FD000904200D110BD441C00B253F8200041F8BB
:103FE000040BE0B2F4E700BF502800400F4B30B59F
:103FF0001C6F240407D41C6F44F400741C671C6FEE
:1040000044F400441C670A4C236843F48073236023
:104010000244084BD2B2904200D130BD441C00B2E1
:1040200051F8045B43F82050E0B2F4E70038024056
:10403000007000405028004007B5012201A900206F
:10404000FFF7C2FF019803B05DF804FB13B5044607
:10405000FFF7F2FFA04205D0012201A90020019440
:10406000FFF7C4FF02B010BD7047000070470000AA
:1040700070470000074B45F255521A6002225A6001
:1040800040F6FF729A604CF6CC421A60024B012255
:104090001A70704700300040CC4C0020034B1B7856
:1040A0001BB1034B4AF6AA221A607047CC4C002081
:1040B00000300040034B1A681AB9034AD2F874283A
:1040C0001A607047C84C002000300240024B4FF08D
:1040D0008072C3F8742870470030024008B5FFF7BB
:1040E000E9FF024B1868C0F3407008BDC84C0020BF
:1040F00008B5FFF7DFFF024B1868C0F3007008BD7A
:10410000C84C002070470000FEE700000A4B0B4837
:104110000B4A90420BD30B4BDA1C121AC11E22F031
:1041200003028B4238BF00220021FDF75DB953F82E
:10413000041B40F8041BECE77050000830520020CC
:10414000305200203052002000F0CAB84FF08043B7
:10415000586A70474FF08043002258631A61022268
:10416000DA6070474FF080430022DA607047000049
:104170004FF0804358637047FEE7000070B51B4B5B
:1041800001630025044686B0586085620E46FFF73D
:10419000B9FA04F11003C4E904334FF0FF33C4E962
:1041A0000635C4E90044A560E562FFF7CFFF2B4662
:1041B0000246C4E9082304F134010D4A2565802331
:1041C0002046FFF7D9FB0123E0600A4A03750092FD
:1041D00072680192B268CDE90223074B6846CDE9C7
:1041E0000435FFF7F1FB06B070BD00BF884C00201E
:1041F000D04E0008D54E000879410008024AD36A23
:104200001843D062704700BF204A00204B684360CB
:104210008B688360CB68C3600B6943614B69036241
:104220008B6943620B6803607047000008B5234B3D
:1042300023481A6942F0FF021A611A6922F0FF024C
:104240001A611A691A6B42F0FF021A631A6D42F082
:10425000FF021A651B4A1B6D1146FFF7D7FF02F1DB
:104260001C0100F58060FFF7D1FF02F1380100F575
:104270008060FFF7CBFF02F1540100F58060FFF78B
:10428000C5FF02F1700100F58060FFF7BFFF02F18A
:104290008C0100F58060FFF7B9FF02F1A80100F57D
:1042A0008060FFF7B3FF02F1C40100F58060FFF703
:1042B000ADFFBDE8084000F08DB800BF00380240F7
:1042C00000000240DC4E000808B500F027FAFFF7B6
:1042D00011FBBDE80840FFF7EDBE0000704700008D
:1042E0000F4B1A6C42F001021A641A6E42F001027E
:1042F0001A660C4A1B6E936843F0010393604FF0FB
:10430000804331229A624FF0FF32DA6200229A61D2
:104310005A63DA605A6001225A611A60704700BF1E
:1043200000380240002004E04FF0804208B51169D7
:10433000D3680B40D9B2C9439B07116107D530231D
:1043400083F31188FFF7FCFA002383F3118808BD7B
:104350001E4B1A6962F0FF021A611A69D2B21A6121
:104360004FF0FF301A695A69586100215A69596142
:104370005A691A6A62F080521A621A6A02F080520E
:104380001A621A6A5A6A58625A6A59625A6A1A6CE6
:1043900042F080521A641A6E42F080521A661A6E07
:1043A0000B4A106840F480701060186F00F4407081
:1043B000B0F5007F1EBF4FF480301867196753684F
:1043C00023F40073536000F07DB900BF0038024051
:1043D000007000403B4B3C4A1A643C4A4FF4404159
:1043E00011601A6842F001021A601A689007FCD541
:1043F0009A6822F003029A60324B9A6812F00C021B
:10440000FBD1196801F0F90119609A601A6842F449
:1044100080321A601A689103FCD55A6F42F001028B
:104420005A67284B5A6F9207FCD5294A5A601A6876
:1044300042F080721A60254A53685804FCD5214B1B
:104440001A689101FCD5234AC3F884201A6842F007
:1044500080621A601A681201FCD51F4A9A60032212
:10446000C3F88C204FF00062C3F894201B4B1A68ED
:104470001B4B9A421B4B21D11B4A11681B4A91428C
:104480001CD140F203121A60164A136803F00F039E
:10449000032BFAD10B4B9A6842F002029A609A6899
:1044A00002F00C02082AFAD15A6C42F480425A6493
:1044B0005A6E42F480425A665B6E704740F2037255
:1044C000E1E700BF00380240000400100070004027
:1044D000081940021030002400948838002004E0BD
:1044E00011640020003C024000ED00E041C20F4199
:1044F000074A08B5536903F00103536123B1054A24
:1045000013680BB150689847BDE80840FFF71EB923
:10451000003C0140D04C0020074A08B5536903F025
:104520000203536123B1054A93680BB1D0689847E1
:10453000BDE80840FFF70AB9003C0140D04C00201C
:10454000074A08B5536903F00403536123B1054AD0
:1045500013690BB150699847BDE80840FFF7F6B8FA
:10456000003C0140D04C0020074A08B5536903F0D5
:104570000803536123B1054A93690BB1D069984789
:10458000BDE80840FFF7E2B8003C0140D04C0020F5
:10459000074A08B5536903F01003536123B1054A74
:1045A000136A0BB1506A9847BDE80840FFF7CEB8D0
:1045B000003C0140D04C0020164B10B55C6904F45F
:1045C00078725A61A30604D5134A936A0BB1D06A74
:1045D0009847600604D5104A136B0BB1506B98478F
:1045E000210604D50C4A936B0BB1D06B9847E205BA
:1045F00004D5094A136C0BB1506C9847A30504D538
:10460000054A936C0BB1D06C9847BDE81040FFF79A
:104610009DB800BF003C0140D04C0020194B10B5A4
:104620005C6904F47C425A61620504D5164A136D34
:104630000BB1506D9847230504D5134A936D0BB108
:10464000D06D9847E00404D50F4A136E0BB1506E3D
:104650009847A10404D50C4A936E0BB1D06E9847CD
:10466000620404D5084A136F0BB1506F98472304B6
:1046700004D5054A936F0BB1D06F9847BDE8104041
:10468000FFF764B8003C0140D04C002008B5034857
:1046900000F010F9BDE80840FFF758B8504D002071
:1046A00008B5034800F006F9BDE80840FFF74EB82A
:1046B000BC4F002008B5FFF737FEBDE80840FFF704
:1046C00045B80000062108B50846FFF769F806213D
:1046D0000720FFF765F806210820FFF761F806219B
:1046E0000920FFF75DF806210A20FFF759F8062197
:1046F0001720FFF755F806212820FFF751F807216A
:104700001C20FFF74DF80C212520FFF749F8BDE8E4
:1047100008400C212620FFF743B8000008B5FFF73A
:1047200017FE00F07BF800F03DF8FFF7D7FDBDE87D
:104730000840FFF709BD00000268436811430160AB
:1047400003B1184770470000143000F0DFB90000D3
:104750004FF0FF33143000F0D9B90000383000F0CA
:1047600055BA00004FF0FF33383000F04FBA000068
:10477000143000F0A5B900004FF0FF31143000F004
:104780009FB90000383000F0FFB900004FF0FF3251
:10479000383000F0F9B90000012914BF6FF01300A0
:1047A0000020704700F060B837B515460E4A026029
:1047B00000224260C0E902220122044602740B4634
:1047C000009000F15C014FF48072143000F04EF95B
:1047D00000942B464FF4807204F5AE7104F138005A
:1047E00000F0C6F903B030BDBC4F000838B5C3694E
:1047F00004460D461BB904210844FFF79DFF2946D6
:1048000004F1140000F040F9002806DA201D4FF4EE
:104810000061BDE83840FFF78FBF38BD0023054A6F
:1048200019460133102BC2E9001102F10802F8D138
:10483000704700BFD04C00200268436811430160FC
:1048400003B1184770470000024AD36843F0C00321
:10485000D360704700100140024AD36843F0C003A0
:10486000D36070470044004010B50A4C0A4A204605
:104870000021FFF799FF094B094AC4E99723094C26
:10488000094A00212046FFF78FFF0849084BC4E979
:10489000971310BD504D00204948000880F0FA02DF
:1048A00000100140BC4F002059480008004400405F
:1048B00040787D012DE9F041D0F85C62F7683368FB
:1048C000DA0504469DB20DD5302383F311884FF4E9
:1048D00080610430FFF7B0FF6FF480733360002312
:1048E00083F31188302383F3118804F1040815F051
:1048F0002F033AD183F31188380615D5290613D52D
:10490000302383F3118804F1380000F065F90028A2
:104910004EDA0821201DFFF78FFF4FF67F733B40D3
:10492000F360002383F311887A0616D56B0614D53D
:10493000302383F31188D4E913239A420AD1236CDC
:1049400043B127F040073F041021201D3F0CFFF723
:1049500073FFF760002383F31188D4F86822D368CB
:1049600043B3BDE8F041106918472B0714D015F088
:10497000080F0CBF00214FF48071E80748BF41F0D9
:104980002001AA0748BF41F040016B0748BF41F032
:1049900080014046FFF750FFAD06736805D594F8D7
:1049A000641220461940FFF721FF3568ADB29EE73B
:1049B0007060B6E7BDE8F081F8B515468268066913
:1049C000AA420B46816938BF8568761AB54204460B
:1049D0000BD218462A46FCF7F5FCA3692B44A361C9
:1049E000A3685B1BA3602846F8BD0CD91846324665
:1049F000FCF7E8FCAF1BE1683A463044FCF7E2FC08
:104A0000E3683B44EBE718462A46FCF7DBFCE36827
:104A1000E5E7000083689342F7B51546044638BFC2
:104A20008568D0E90460361AB5420BD22A46FCF7F5
:104A3000C9FC63692B446361A36828465B1BA360C0
:104A400003B0F0BD0DD932460191FCF7BBFC0199D2
:104A5000E068AF1B3A463144FCF7B4FCE3683B44E2
:104A6000E9E72A46FCF7AEFCE368E4E710B50A4440
:104A70000024C361029B8460C0E90000C0E9051105
:104A8000C1600261036210BD08B5D0E905329342EE
:104A900001D1826882B98268013282605A1C426107
:104AA0001970D0E904329A4224BFC36843610021DF
:104AB000FEF7BCFF002008BD4FF0FF30FBE7000011
:104AC00070B5302304460E4683F31188A568A5B15E
:104AD000A368A269013BA360531CA36115782269F6
:104AE000934224BFE368A361E3690BB12046984772
:104AF000002383F31188284607E031462046FEF75D
:104B000085FF0028E2DA85F3118870BD2DE9F74FA3
:104B100004460E4617469846D0F81C904FF0300ACF
:104B20008AF311884FF0000B154665B12A463146CD
:104B30002046FFF741FF034660B941462046FEF795
:104B400065FF0028F1D0002383F31188781B03B0A0
:104B5000BDE8F08FB9F1000F03D001902046C8479F
:104B6000019B8BF31188ED1A1E448AF31188DCE750
:104B7000C0E90511C160C3611144009B8260C0E9B6
:104B80000000016103627047F8B504460D46164601
:104B9000302383F31188A768A7B1A368013BA36002
:104BA00063695A1C62611D70D4E904329A4224BFC1
:104BB000E3686361E3690BB120469847002080F306
:104BC000118807E031462046FEF720FF0028E2DA90
:104BD00087F31188F8BD0000D0E905239A4210B58B
:104BE00001D182687AB98268013282605A1C82617E
:104BF0001C7803699A4224BFC36883610021FEF7D1
:104C000015FF204610BD4FF0FF30FBE72DE9F74FB1
:104C100004460E4617469846D0F81C904FF0300ACE
:104C20008AF311884FF0000B154665B12A463146CC
:104C30002046FFF7EFFE034660B941462046FEF7E7
:104C4000E5FE0028F1D0002383F31188781B03B020
:104C5000BDE8F08FB9F1000F03D001902046C8479E
:104C6000019B8BF31188ED1A1E448AF31188DCE74F
:104C70000B460146184600F02DB8000000F040B881
:104C8000012838BF012010B50446204600F030F856
:104C900030B900F007F808B900F00CF88047F4E7E5
:104CA00010BD0000024B1868BFF35B8F704700BF58
:104CB0002852002008B5062000F084F80120FEF7F5
:104CC000EDFF0000024B0A4601461868FFF720B9C5
:104CD0001C23002010B5054C13462CB10A46014692
:104CE0000220AFF3008010BD2046FCE7000000006A
:104CF000024B01461868FFF70FB900BF1C230020C4
:104D0000024B01461868FFF70BB900BF1C230020B7
:104D100010B501390244904201D1002005E003782A
:104D200011F8014FA34201D0181B10BD0130F2E76A
:104D30002DE9F041A3B1C91A17780144044603F1E3
:104D4000FF3C8C42204601D9002009E00578BD4295
:104D500004F10104F5D10CEB0405D618A54201D1EC
:104D6000BDE8F08115F8018D16F801EDF045F5D09C
:104D7000E7E700001F2938B504460D4604D916237D
:104D800003604FF0FF3038BD426C12B152F8213051
:104D90004BB9204600F030F82A4601462046BDE8CF
:104DA000384000F017B8012B0AD0591C03D1162344
:104DB00003600120E7E7002442F825402846984791
:104DC0000020E0E7024B01461868FFF7D3BF00BFA1
:104DD0001C23002038B5074D002304460846114621
:104DE0002B60FEF75FFF431C02D12B6803B12360E9
:104DF00038BD00BF2C520020FEF74EBF034611F80D
:104E0000012B03F8012B002AF9D170476F72672E2E
:104E10006172647570696C6F742E435541565F47BB
:104E20005053000040A2E4F1646891060041A3E5FC
:104E3000F2656992070000004261642043414E49D7
:104E40006661636520696E6465782E0080000000ED
:104E50000080000000008000000000000000000052
:104E6000551C00083D2400089D230008651C00080F
:104E7000991C0008951E0008691C0008791C000890
:104E80006D1C0008751C0008711C0008BD1D000881
:104E90007D1C0008092700088D1C0008911D0008D2
:104EA00063300000A04E0008784A0020884C0020A3
:104EB00000400000004000000040000000400000F2
:104EC00000000100000002000000020000000200DB
:104ED0006D61696E0069646C65000000A0011028B6
:104EE00000000000AAAAAAAA50011024FFFF000097
:104EF000007700000000000000A40A01000000008C
:104F0000AAA6AAAA80500000DFEF000000000077E8
:104F1000880000000000000000000000AAAAAAAA61
:104F200000000000FFFF0000000000000000000083
:104F30000000000000000000AAAAAAAA00000000C9
:104F4000FFFF000000000000000000000000000063
:104F500000000000AAAAAAAA00000000FFFF0000AB
:104F60000000000000000000000000000000000041
:104F7000AAAAAAAA00000000FFFF0000000000008B
:104F8000000000000000000000000000AAAAAAAA79
:104F900000000000FFFF0000000000000000000013
:104FA00000000000000000000A00000000000000F7
:104FB00003000000000000000000000000000000EE
:104FC00065470008514700088D47000879470008E9
:104FD00085470008714700085D47000849470008F9
:104FE000994700083CB2FF7F01000000000000006C
:104FF000E9030000000000000000070000000000BE
:1050000040420F00FE2A0100D204000020230020AD
:105010000000000000000000000000000000000090
:105020000000000000000000000000000000000080
:105030000000000000000000000000000000000070
:105040000000000000000000000000000000000060
:105050000000000000000000000000000000000050
:105060000000000000000000000000000000000040
:00000001FF
